:020000040009F1
:280000000108006999994204204EB1FD0400FFFFFFFF4006000000A0027020020A00280009000000000000001D
:FB002800411A0042726F6164636F6D20426C7565746F6F74682044657669636500980100034C30003003420043004D00390032003000370030003200200042006C007500650074006F006F0074006800200034002E0030005C0100017A020000089304002000000068040012000C00920600A300C80014646A3600038011000000B0000000A0000000420000005200000080000000900000006200000072000000C0000000D0000000220000003200000069020003015D0C000A64E6B000008898425A33435F09003C280100040004F70C0A6F0098160800C600F3025D0066033000C900E10268005C033600C300E2026A0053033C00C200E1026C004E034109
:FB01230000C500D60272004A034300C300CE02790042034800C500C00283003A034E00C800BF0282003B034E00C900BC028400370352000808070707070707060606060505050502C0E40094FC0E00FFFF00005E02000030FC0E00FFFF0F006304000000FD0E00FFFF0F006602000088FC0E00FFFF0000000400002CFC0E00FFFF00004904000070FC0E00FFFF00000B09000074FC0E00FFFF00002E010000D8FF0E00FFFF000062190000D0FC0E00FFFF000020C90000C8FC0E00FFFF000038850000DCFC0E00FFFF00001CC80000CCFD0E00FFFF0000048000005CFC0E00FFFF00000200000020FC0E00FFFF000019210000E0FC0E00008000000000000065
:FB021E00C0FC0E00FFFF000022000000948F0800FFFFFFFF00100010988F0800FFFF0000001000009C8F080000FFFFFF000A0A0AC3160012691418310870007836042430607180764A3108290ACF0900100F0C6EF0B009F0601A2400FF0108080A10060E020CFE0AFA08F606F204EE020A10060E020CFE0AFA08F606F204EE020301000182D600FF0602020A233C5A6E7D80008000800080008000800080028002800280028002800214FF18880AFF200000000000000000000000000014FF18820AFF430000000000000000000000000014FF18000AFF660000000000000000000000000014FF18080AFF660000000000000000000000000014FF180B0AFF05
:FB031900430000000000000000000000000014FF18100AFF200000000000000000000000000041000000007B0000000041000000007B0000000041000000007B0000000041000000007B0000000041000000007B0000000041000000007B000000008612000413004008000040130001000180FF000113C15E0044041422A244041422A23B04B104B204B304B404B504B604B704B804B904BA04BB04BC04BD04BE04BF04C004C104C204C304C404C504C604C704C804C904CA04CB04CC04CD04CE04CF04D004D104D204D304D404D504D604D704D8280C000B0400B64B09000B0400604C09000B0400324D0900081F0000B0DB010078F0ECFB10008C6309005B
:FB041400281C5F3000210170391C321D87F70CFC080F000184E0000030BD00B50000000000000817000288E0000087F0CEF808002852090000F002F800BD000008170003586600008FF04CF90800F4580900FFF793FF30BD00000B04008E5A09000B0400B85A090008170004209E02006CF0C2F80800A85F0900FFF7C0FF70BD000008150005C08400008DF0CEFD060060600900FFF7A6FF30BD082D0006B47702006EF057FC1E006660090002B461684907C90F301C91F727FD02BC002902D0F06991F79CFB91F79EFB080F000724B500000FE0C046000000000000080F0008C44F000010E0C046000000000000086700091CF0030057F032F8580084600968
:FB050F000070B5061C0C1C151C002B21D104A8008840281DD105A80088202819D15A2917D8081C15D003F016F9002811D1032D0FD02204121408210748002303F013F9002806D1221C291C301CA9F765F8012000E0002070BD18650800080F000A988000005808042B0000000000000817000B680C040055F038FA0800DC60090000F002F870BD00000819000C64D4000088F0BCFE0A00E0610900281CFEF7BDFF77F752F90813000D08D6000088F0EFFD0400EA61090077F710FA080F000E80DA0000C046C0460000000000000815000F2452000090F0E3FF0600EE61090000F001F8F0BD0B04005063090008190010845C020070F08AFB0A009C6309009B1E
:FB060A00005859EF188FF771FC0815001164F8000086F09FFD0600A663090000F001F8F0BD081700128002030066F052F908002865090000F09AF899F7CFFE081700132848020071F082FE08003065090000F03EFA8EF7D5F908170014B473020070F098F90800E8760900FFF770FE8FF7F3FE080F001534C40100C046201C000000000000081700161403030067F0ECF90800F0760900FEF7ECFF6CF75CFE081700172447020071F008FF08003865090000F0CFF98EF707F9081700186847020071F0EAFE08004065090000F0E1F98EF71FF9081700190C4D020071F01CFC08004865090000F06EFA8EF7F6FB0817001A404D020071F006FC0800506509001C
:FB07050000F084FA8EF710FC0817001B7C4D020071F0ECFB08005865090000F0EEFB8EF724FC0817001C7854020072F02EF90800D8760900FFF7CAFD8DF7DDFE0817001D0C57020071F0E8FF0800E0760900FFF726FE8EF760F80869011EA444000093F0ABFB5A01FE7B090000B526490B6824490B6022490B6820490B601C490B682B490B60414B42490B6033490B680120C00303430B603F490B78002B04D02E490B68400303430B602B4A13685B085B001360394B394A1360B1F785FBB1F7AEFFB2F7FDFAB2F7A3FC0D21354801F04AFB344A9068002803D099F7AEFCB1F74AFA2148264A60E0C046C0B00800FFF2011AD4940900848FB002D08B0E00A06F
:FB080000800E00D8940900148B0E00DC9409006CE50500E09409008C150800DF7A0900237B0900EF7B09006B7B0900D77B09005C000F0094830E00FF00FFFF608B0E0040230001E08A0E00E02C0800A4860E0088B2080005000080850000801C800E0014800E00848F080004830E00CCFC0E00F893090000940900FC930900108B0E00C42C0800CC2C0800D02C0800BC8B0E00AD020000CC8B0E001CCD080010325476D48B0E00009D0800ECCC080013680360034A11680161034A1168416000BDC046CC2C0800D02C08000861001F0044000093F0F2FA5200E879090010B5A448002383700423437001230370A14BA2480360A24BA24C2360A24C2368A24C3F
:FB08FB002360A24C2368A24C23602C22A249A248BCF7B3FFA148A14C2060A149C160A1494162A1490161A14B8361A14BC36110BD080F0020D0B80400A5F809E00000000000000815002120BA04004CF0FEFB060020820900FFF7D4FF30BD081500223CB004004DF0F3F806002682090000F001F870BD08170023EC8A04004FF0DEFB0800AC82090000F002F8F0BD0000081700243069040051F088FD080044840900FFF7C4FFAEF790FA08190025545D040052F07AFB0A004C840900B4F708FDFFF7B2FF30BD08190026E0A504004DF039FF0A005684090000F003F803B0F0BD000008170027E882040050F008F90800FC84090000F002F830BD00000817001E
:FB09F60028B0B104004DF01EFA0800F085090000F002F830BD0000082B0029DCC004004CF0EAFA1C00B4860900FF233D3343430448C0189F300078002800D101207047C046349D0800081B002A94AC04004DF026FD0C00E4860900201C00F003F8B2F7D6FA0000081B002BACAC04004DF066FD0C007C870900201C00F003F8B2F796FA00000823002C3CC104004CF0C8FA1400D086090029187F231B02FF339D4200D35D1EFF23B3F72EFD0817002D981B030066F068FE08006C880900FFF7D2FF30BD0000082B002E1C7B040050F0C2FE1C00A488090004910FB4301CFFF7E3FF012802D10FBC05B0F0BD0FBC062DAFF730F9081F002F18AC04004DF08EFE0B
:FB0AF10010003889090003D1FFF7C1FFB2F76EF9B2F76DF90000081700306CA804004EF0A6F90800BC8B0900FFF74CFFF0BD0000088F0031D8F1010079F0F4FC8000C48B0900F0B583B0012100910027C0237B431A481C18206BC00729D5251CBC356B78002B24D1261CE38D2C36002B1FD0B379002B02D00021009119E0211C0C310F48052200F058FB002811D00223B371201CB3F7F6FA01A9201CB3F7DEFA01A9A878B2F778FB082201A9A878B3F7FAFB01370F2FCBD3009803B0F0BD28900800104F0800087700327461030062F066FD6800448C090010B500248DF73AFA012803D309D0022820D102E09FF784FE01E0A5F7ECF9041C18E00D490B7800F3
:FB0BEC002B14D00C4A106803680B4A13600B4A1378002B0BD08B784978002B03D04B00FF21013101E04B00802199400160201C10BD481B0800E40A0800AC5808003A010800080F00337C640200131C036000000000000008570034B462020072F0FAFC4800AC8C090000B50D490868002804D003280FD0052811D104E009480378002B0CD007E0084B1868012200219AF756FD9DF728F905490B680120186000BDB0C80800D1CA0800F40A0800E40A080008230035C0B903005DF098F91400F48C090003D100F007F8012802D0A000A2F760FEA2F760FE081900367847000094F04AFC0A0010900900381CFBF7A1FE6BF7B2FB08190037AC47000094F035FC71
:FB0CE7000A001A900900281CFBF7BAFE6BF7CBFB081B00383CDB00008BF072FA0C002490090081B000F003F874F7ECFD000008270039405B010083F0ECF818001C8D0900002E02D00020E05504E0E35D002B01D0013BE3557CF71FFF081B003A50A704004EF078F90C00448A0900381CFFF795F902B0B1F782FE0817003B58A704004EF07AF90800508A0900FFF7B3F9B1F78FFE0821003CB03C010085F034FA12001C91090001B4301C00F010F801BC75F7CDFF7AF7C3FD081D003D5CB503005DF0E7FD0E002E91090001B400F00FF820BC6B01A2F712FA0817003EA8A003005FF048F808003C91090000F015F8A0F7CEFF082B003FCCB203005DF064FF1C7B
:E60DE20000989109001378002B07D103B400F008F8012803BC01D1A2F792F8A2F79CF80000081B004074B403005DF0AAFE0C00CC91090000232B7500F02CF8A2F750F9081D00411C69020072F05CFC0E00D891090003D100F027F8A3F703FB8DF79EFB0827004230BB03005DF059FB1800E6910900012D03D1002E01D100F056F8A068A3F71EFA0021A2F79CFC082700430862020072F0F9FF1800FE910900201C08B4019900F01BF808BC9C4201D08CF7FDFF8DF707F8082500449CBC03005DF0BBFA1600169209001B0705D400F044F8002801D1A2F73DFDA2F768FD00000A05002DCB080001FE0000E2
:FB4B000030B530483049086030483149086000F01BF901F0CFFC00F03BFB00F04FF900F0FFFA00232B48037000F05AFA00F06CFA03F012F92849081CE430284B0360284D2B6802252B43264D2B60264A13688024A34313600023244D2B70244B244D2B60244B254D2B60254B254D2B60254B264D2B60264B264D2B60264B274D2B601223264D2B70264B274D2B60274B274D2B60274B284D2B60284B284D2B60284B294D2B60294BCB620023284D2B60284B436530BC08BC184727482749086027480649C8647047B1510900BCC80800B5510900F0C4080054960900A0190800515209006C010F0040150800FD07080041450000F893090020C90000FC930923
:FB4BFB00001CC800000094090062160000D8FF0E0042050000881308006C0400008C130800901308002F450000781308000EC90000801308000AC800007C1308001E45000084130800268500007413080049890900F49309009D640900014B0900900008001563090070B500200F49104B4B6114E06B099C00EB06DB0E01259D400B592B430B5143004C69C50052195268012632432725AD03AA1A1A530130054AC3009D58922DE5D370BDC0464C1B0800389509004893090030B582781202437813439A05920D1B0AFC252B400C2B05D1032A2ED104F067F801202BE00124FC2B22D1C22A0ED0C32A0FD0C62A1ED30FD0C82A10D312D0CB2A13D9E62A16D1FC
:FB4CF60003F0CBF914E001F014FDE6E701F05AFDE3E704F07BF8E0E704F0B5F8DDE704F0F2F8DAE796F789FDD7E7042B02D10024201C00E0002030BC08BC18470248024908607047C046B14C090018C90800002070470148024988607047454D0900201A080030B5051C7AF7B2F9041C281C8AF741FA8749201C2830062204F0A2FA00280BD1844C2560012363717F21C943A01D072204F09EFA00232371002030BD10B5041C0120A040C1437C4803680B40036089F775F978480368A34203D1FF2303600023437110BD75487649C8607047F0B583B0041C012906D164300023C372251C9435AB73EB736F4803689B079B0F032B02D071F780FAC8E00023A35C
:FB4DF10081E07B484000D1B6E070F71BFD002803D1674803691B0101D5012100E00021271C64373E1CFB6880208343C8010343F3600C365F4A1078431006D0C3071B0E31688020814319433160594803691B0102D4381C94F7F8F9BB69002B02D03B681B063BD4338868460380E37B012B0DD0251C94356B7B002B10D02B88042B0DD3EB7C022B0AD3AB7D002B07D1A72303201855009B78208343002106E00121E974009B78208343082003431F20800283438802034300931B041B0C3F4A1360012030723B4A13691B0152D400984006010F00231A1C012094F7D8FB45E0E07B002802D1A72301221A55012804D1E37C042B01D072F7CBFCF37A002B06D0FC
:FB4EEC000023F372336801204002434033600121B172251C9435A97326480369DB0002D5201C87F7DBFD338824490B60B0884860381C70F7FBFC30684006030F2048C05C3072431EA381E37B002B0FD10121387F81401C4A1068084008D1E37C042B05D019480378AB7519480378EB75114803691B010FD5201C94F731FF0BE0271C64373B727B7270F789FC636C002B02D05A231B5BA38103B0F0BC08BC184709C108000494090000040800C54D090000020800188B0E0054200800DCC80800CC8A0E009EBB0500B4010800F5010800F601080030B50D1C041C75F7CFFE6B075B0F012B05D1E37B002B02D1A07B9CF70EFE30BC08BC184700B52C2204490521
:FB4FE70048BFF7CCFC034804494161044B186000BD0CBD050014940900BD4F0900E402080010B53F4C3F4B1C602C223F49201CBFF7B5FC3E48606210BDF0B5041C051C876A28353B4B42331878002866D1201C012172F729FA061E4BDD022804DB201C77F7A3FA002859D1618C8B1F9E4223DA304A13689C420BD0391CAB310878013800D30870731C5910201C77F730F830E0731C5810E37B002B05D07B6C002B02D06B7F002B25D02F89B84222D36A89002A06D1A389002B03D1201C71F737FE18E0BA4200DA3A1C904201D90C2310E04B23A27C1B5D9A420CD102280AD36B7F002B05D014480378994201D9282300E03823A374211C4D31087800280FD0D4
:FB50E2000238087000060BD1E37B012B02D0237D0C2B05D0321C201C0523022177F78CF9F0BC08BC1847409409000003080074BD0500215009006C210800F402080000B52C2216491748BFF72CFC1548164B18601649016100BD30B50D1C041C78F774F8022D09D16B23185D002805D0201C87F75DFB201C87F795FB30BC08BC184700B5011C6831CB78002B07D04B7A002B04D18B78002B01D087F76CFB00BDC0462CBE05006C940900300308003951090000B52C2203490448BFF7F4FB024B0348036000BDB0CB050098940900F40308000020704730B5041C002921D001291BD1400511D41CE0124D291C1248B8F737F82988281C262902D103F023F904DF
:4B51DD00E089000D4A8958C6F767FB0A48B8F740F80028E9D00A4B1C4003E0022901D17CF745F8201C30BC08BC18470548064908607047F4440800284508009CBE0500FFFBFFFFB5510900F0C408008F
:FB52300000B5431E04490B6004490B78032B01D1C0F762F800BDC046E08A0E0038080800F0B587B0061C0491081C00210391A94C2064211C4431009100238B70A6488568002D00D121E2AB7D002B09D0012203920023AB756361237810208343237006E06069002803D0012E01D970F77BFF22691D27FF03002A50D0607A012803D19389002B4AD047E0954B1B5C002B43D1BB68DB0742D4137D092B3DD204281AD1012E18D196756261237810200343237023683B608B490B687233187802282DD0002388490B608849086888490B6803600B68036022E002280AD1012E08D196756261237810200343237023683B6015E0032803D17F498B78022B0FD0068F
:FB532B002801D0032805D1012E03D1BB689B0600D573E1122803D0102801D070F7A5FE704B985D029000284AD00123DB0733430193714B724908689863714901220A600099CB78012B30D06F490B689B0C9B040B600B686D49086803436A490B600099CA706A490B686A490B606A490B686A490B606A490B686A490B606A490B686A490B606A490B686A490B606A490B686A490B606A490B686A490B606A490B6856490B606949086869490860A87B2318042801D3187800E0205C6F229043187050E0A87B225C0F218A433107090F0A43225423180428049802D38107101C01E081071878490E6022904308431870434B584908689863009AD378002B30D0FF
:FB54260042490B689B0C9B040B600B685349086803433D490B600023D37050490B683D490B604F490B683D490B604E490B683D490B604D490B683D490B604C490B683D490B604B490B683D490B604A490B683D490B6049490B6829490B60484908683C490860002101912868826A281C0021C6F70CFA002810D026231A5C002A0CD08368002B09D00298002804D0802301981843019001E0012200E00022237880208343D0010343237020200499084001D00120C003334908600499090704D432490B68802083430B600499880801214140A27880208243C8010243A27056E0C046642C08006C210800ECBB0500DC02080060000F00AC2C0800440208008807
:FB5521002B08002CFC0E0060020800E08A0E00B88A0E005C0208006C130800D8FC0E0070130800E0FC0E0078130800CCFC0E0074130800C8FC0E007C130800DCFC0E0080130800D0FC0E0084130800D4FF0E00881308008C13080030FC0E00B82C080048020800BC2C0800C02C0800C42C0800C82C0800CC2C0800D02C0800D42C0800D82C0800DC2C0800648B0E00A4860E002868826A281C0321C6F77AF9AD490B78012B01D077F71AF905A9AB4A13687020034018099CF767F92369002B14D0637A032B11D188F7C8FC002806D1A3480368032B02D00368062B06D12B7C122B03D100980121817058E005988007800F06D003280ED1069B9A4908888342D3
:FB561C0009D30398012800D1656170F735FD009901224A7043E00820B860A87B786223683B603B1C1833221D03929207920F02D1039909680FE00399891A0391D2000968D140049120218A1A03994968914001B40598014301BC1960BA69331C103B042B0DD2FF23013383407F4810401843B861102E07D17D4908687D49086002E07A481040B8610198002800D07861E5602672002300990B704B70281C8CF77CFD012007B0F0BC08BC1847F0B5724CE568002D02D1201C0930A0E0EB7B012B09D1201C1830AB7BD90043586B4A13600B185B685360217A694F3868012901D1084301E04008400038602868826A281C0021C6F7D1F800281AD02623195C0045
:FB5717002916D08368002B13D070F76CFF5D4E237AF05C5D490B68002803D001204006034320E05A4803400B603B6802210B4318E055490B68554803400B60524E237AF05C002802D05249887901E052490868236CDB0601D4504908603023DB432E3338680340391C0B602868826A281C0121C6F793F8071E12D00368002B0FD04749086900010BD41022391D4548BFF7EFF8386844490B6883210B40184303E0414A1068832108403F490860207A335C3E4A002B136814D0012189030B4313603B490B683B490B403B490A78520213433A4E33603A4E33683026B3431021194308E038490B401360314A1368334A1360334A1168344A116060720023E360A4
:E2581200201C0830256100220270F0BD10B51B4C1E4B607A185C002802D070F7A2FF15E06069002801D070F7ACFC28490868637A012B01D1274A00E0274A13680360116801600023254A136070F7B7FE002323490B60E3602361637244340120207010BDC046D4C1080024860E001C840E00E4B60800FFF0FFFF9406080064FC0E00642C080018820E00A8860E00ECBB05001C800E00FFFFFFFD002D08007C030800108B0E005420080080810E00E88A0E00808B0E00B02C0800FFC1FFFF9013080088FC0E00B42C0800FFBFFFFFCCFD0E00AC2C0800400208004402080060000F0018800E0007
:FB58FC0070B582B0061C65480168890602D5022072F765FC624C2568A3682360002D26D0002E18D19EF73AFA002814D0C30703D52A68916900290BD1430703D52A68D169002905D1830706D52A68116A002902D0281CC5F7B2FF9EF73EFA011C2A685269002A04D0002802D0281CC5F7A3FFA0680026A84218D0002D21D02A681269002A03D0281C0521C5F795FFAE8123699D4200D126612B7D092B11D3281C73F72EFE281C73F7B3F90AE0002808D06369984205D166613B4800220121B7F763FF3A48C16E002904D0A368002B01D1C5F775FFFFF77AFEA06800284BD08681037D092B20D26369984205D166612E4800220121B7F748FFA068A84206D10115
:FB59F700684968002902D00523037508E0017D032901D0042905D101684968002901D0C5F74EFFA0680223037501680A69002A02D00221C5F741FFA068807B1D4A136870210B401909884216D169469BF730FF70F7A6FC002801D0174800E01748028800998907890F04D0032905D1019B934202D33F2301201855A0688CF726FA01208CF736FAA66066603C3426716671012002B070BC08BC18470948044988617047C046C4C408006C2108000C2D0800201A080024860E006602080064020800FD580900A248A3498865704700B5A24A9007800F01D1116808E0121AC0001368C3402021081A516881401943C90F9B4801709B4A1068002817D09A4A0260C7
:FB5AF2009A4A82609A4AC2600123994A13700023994A1360994A1360994A1360012902D100F007F802E04068C5F7CBFE08BC1847000000B500F003F808BC1847000010B564238F48037000238F4803608F4803608F4C236000F04FF8804A9007800F01D1116808E0121AC0001368C3402021081A51688140194301204007014015D084490B68001403430B6083490B68834803400B6004390B680120800303430B607F4B80490B6003037F490B606B4A9007800F01D1116808E0121AC0001368C3402021081A516881401943C90011D5774C2368002B02D0201CB7F74BFC7449201C00231A1CB7F726FC72480168201CB7F72CFC8EF7A8FA10BD10B56F4C2384
:FB5BED0068012423436D4C236001239B036C4C2360534A9007800F01D1116808E0121AC0001368C3402021081A516881401943090105D561480368022003435F480360604800218160F421C16020210161E8218161E9214161102141624021C161016205239B04036010BDF0B582B0041C01910B1C0026009653490F683F0C3F045B0051481D5A51498D4211D180231A5D5048135C1B014F4818188388002B07D04B4D1035837A012B06D1484D203503E0002D01D12E1CBEE0201C8CF70AFC002800D0402545480368002B07D0602D01D1E0251BE0702D08D1D02517E00198042801D0022801D101263604302D06D17023185D002802D0354D703507E0502DCD
:FB5CE80005D1236FDB0502D501235B041E432E432F4B70339D4203D02B093148C15C0091302D0BD17023185D002807D1201C2830037D807A19180906090E0091009803031E43E37B002B02D00123DB031F43E37C032B49D1608CC306180F43E0C15A0900A0190800C005080030C8080044060800255B0900555C09002F5E0900B805080034C8080038C808003CC80800D005080040C8080048C808004CC808009C800E0010800E00FFBFFFFFFF030000BC820E0010000C0068500800673D0200D405080070010F005C000F0074820E00D8050800100100009005080024500800D4C408002406080003021F43402D25D14B480378002B06D0201C8DF7E7FE0327
:FB5DE300071B0A1E431AE00123DB041E43A07B9BF772FD4008434A1060434A11689BF706FD424A1060424A1368984204D2201C8DF7ADFE002802D00123394803703D480660476002B0F0BC08BC1847F0B582B00F1C051C0022009201908CF73EFB354E002844D034682E48017800291AD1A87B9BF742FD40082B4A10602B4A11689BF7D6FC2A4A10602A4A1368984204D2281C8DF77DFE00281BD0012321480370264B1C4015E06B6E1B0612D4012910D1281C8DF76DFE00280BD1A87B9BF71DFD41081A4A11600023164A13700123DB041C4314480378002B03D001988CF7A7FF0090174B1C40009803071B0A1C433460042F01D0022F05D133680121090420
:CA5EDE000B43012107E00F480378002B06D033680E490B40002133600B48017002B0F0BC08BC1847C046B805080038C8080034C808003CC80800CC05080070820E00FFFFF7FFFFFF0FFF45C80800FFFFFEFF70B503685A06120F092A04D0847F9B05DB0FA34204D0C368144C2343C36012E04B03C36806D4114CA343C3600823104D2B7008E00D4D2B43C36001236340837705230B4E33700B4C23680133012B04D0082A02D10123084A137002234372436804221343436078F77CF870BD00010000E8C00800E08A0E00EAC0080033
:B05FB00030B5041CC37C032B27D1037D0C2B24D11830437B002B20D121490B699C4202D18B68002B13D0418900680B1858010509A07B9BF77AFC854201D3281A03E0431B01200007C01A831F1648834205D3201C73F7FAFA201C72F788FF237D022B03D0032B01D0042B07D10F480379002B16D0201C70F7D1FD12E00C480369002B02D0201C70F766F806494123585C012804D0002804D10B689C4201D172F7F4FA30BD6C210800FBFFFF07A42C0800642C08009F
:FB60E40070B5041C00253848436912219B0708D5364A1068364A106050304079122800D8011C43209DF79EF8324BA360324B2361201C0830AAF73FFF2168086063681D60AAF7A8FF201C1030AAF735FF216808600420AAF7B7FF6061062801DAAAF79AFF201C0830AAF727FF216808606368002018600420AAF7A6FFE060201C1030AAF71AFF216808606368002018600420AAF799FF6061E368C61A301CAAF7E9FF042817DD01350C2D14D0301C042E08DDAAF7DFFF8100081A2169081802382061CFE7AAF7D6FF8100081AA168081A0230A060C6E7A16820690B1AE3614018C30F18184310236270BDC046181B0800D4CC08001C960900FF03000001FCFF73
:0161DF00FFC0
:FB61F400F0B5444D2B68987B9BF76DFB46082B68996C301C9BF702FB041C2868011C94314A88002A10D094420ED9037D0B2B0BD00D2B09D070F7D1FB2B686433197F012000037BF7A3F864E00B7D002B06D0CB88F31A1B041B0C9C4200D81C1CC36F6430002B06D00B89F31A1B041B0C9C4200D81C1C8A88B31A1A04120C944200D8141C0B881F1FBA4204D3CB7C022B01D30023CB74214E33889C4204D80020BA422ED303202CE073889C4201D8042228E0B3889C420BD9007F74F7F3FE002814D0037C112B11D115494B889C4203D829689431052215E08B889C420DD82968943106224A745E2383740CE0F3889C4203D829689431062204E029689431078C
:AD62EF002200E0021C4A740B7E012B04D1531F012B01D804234B74F0BDB421080034020800EC02080010B5A3F705FC0B494B699B070FD50A48036801200343084803600A249BF782FD013CFBD1044803685B085B00036010BC08BC1847181B0800F0FC0E0010B5094C2C220949201CBEF713FB0849E160084B1C6010BDC27B4A4002D0838C05490B607047C0462096090034CC05006963090010040800CC8A0E00281C5F3000210170391C321D87F70CFCC9
:FB63AC00F0B5041C0027C56D8726F600002D04D1301C9BF7DEF8051E03D0301C9BF7D9F8071C2E4803689B025B0F012B2CD1A9F7AFF9002828D02A480368002B09D1301C08309BF7C6F8264A1060311C0831BEF7E5FD24480368002B09D1301C08309BF7B8F8204A1060311C0831BEF7D7FD002D0ED0002F0CD01B480368002B08D018480368002B04D01BE0002D01D0002F17D1E02300201851E565E4210859C30208D4031C114803430B515022206807217DF7FEFA0E480368002B0DD19BF796F80AE0E5656760E4221359074883431351206807217DF70DFB0020F0BDC0464C0B0800444408009C440800000010006003080000231360012805D10123DB05
:8164A700040B6007239B031360704700000C480D4908600D480D4908600D480E4908600E4B0E490B600E4B0F490B600F4B0F490B600F4B10490B60104B10490B607047C046336C090064C808009D6A090068C808001970090080C80800E165090054C808008968090070C8080031750900509609009970090078C8080070930900B006080017
:FB65600070B5051C7CF771FA011C041CEA691204D20F2273032363730C34324B186800090226800706D5F42043599B0702D5A6702D480660F4204359DB0601D4002A01D1002000E029484860281C90F702FF0023274A137070BD30B5041C0D1C7CF745FA24494B681A7BD207D20F0273052343738573214A4260011C201C90F7EAFE30BD70B5051CF4352B68DB0603D50321FFF7E2FF1EE0061CAC68002C03D0201CB6F730FF0AE014209AF785FF041E11D0A860321C12490023B6F705FFF1690906C90E201C0A2902D1FF21913100E01021B6F704FF08494B68987B0349086070BC08BC1847C046641B080088500800D34902005CC80800F4440800F96C09D3
:FB665B0000D345020010B5041C6B4A1068C00702D4112323702BE008790002C9780843012178F7ABFA002803D0F8221158490701D51223EEE7C169090403D4F4210B589B060DD55D4B19684906490FF42212589207920F914203D159490B78002B01D00C23D7E701230B7028342370FFF74BFF10BD30B5051C0C1C08790002C9780843012178F77BFA002805D0F8221158490701D40B2019E0C169090417D4F43003685B0601D40E2010E0282301205855424908684006400F022808D1414A1188601D01F0DDF8002801D10D20287030BD30B58A7B002A01D1122340E0374CCB7820680225002B06D0012318432060364803682B4305E001239843206032481E
:FB6756000368AB43036031480B7903704B7943708B7983702F48CB79202B02D12E4B186002E02D48402BF9D0487A00020B7A184340102A4B1860C0006080C87A00028B7A1843204B1880487B00020B7B1843244B188024480280CB7B244803700B7C2348037030BD164A1168C907C90F817317490B78C3734B7803748B784374164A1168090A8174164A11684900C174090A01750D4A11884175090A8175114A1188C175090A017610490B8843760F490B7883760F490B78C3760E23C3707047C046641B08005CC80800E8930900301B0800A80608001E200000940608003A40000090060800EA930900EC9309004D9609004E96090010B5041CFF20052194EE
:FB685100F7B9F9002806D016238370C470210A017194F73BF910BD10B5041CFF20052194F7A9F9002806D018238370C470210A017194F72BF910BD10B50024201C00F0A9FB0134042CF9D31821B048BEF794FB00F02AFFAE480268D10708D55106490F022904D1AB4A116872230B4313600023A9490B70A9490B704088C010A8490860A8490B7010BC08BC184730B5051C002429236343A4481818811C281C062202F0E3FC002803D1201C00F074FB02E00134042CEDD330BD00B50021292048439A4A8218507800021278104302D08DF718FF04E001310429F0D38EF74BF800BDF0B5061C04250024904F29206043C019811C301C2830062202F0B7FC0028B1
:FB694C0001D1251C02E00134042CEED3042D0DD1002429206043C119487800020978084301D1251C02E00134042CF2D3042D18D229236B43DC19311C2831A01C0622BDF7FBFF5C20805B2070000A6070311C201C083000F008FA311C283175480622BDF7EBFFF0BDF0B5041C0F1C0026292070436E4BC518A91C381C062202F077FC002803D00136042EF1D326E0201C78F7C1FC291C0831201C00F075FAE0690F21C9050843E061201C0F2303863030868D69780C022A781443A64205D05E4A0121B14013688B4313605B4A0123A3401168194311608485012000E00020F0BD10B582B0062255496846BDF7A7FF002469460623634347481818062202F0386C
:FB6A4700FC002801D0012003E00134042CF0D3002002B010BDF0B582B0071C062248496846BDF78CFF00243B4E0622151C65436946A81902F01DFC002806D1391CA8190622BDF77CFF012003E00134042CEBD3002002B0F0BDF0B582B0041C0E1C171C394DFF2001302058002801D0B6F7D6FCF8210859C00700D48FE0002E00D18CE0002F00D1A3E00859800700D49FE00026E069000408D501A886706846831D2A480122002194F7A3FA201C6DF7F8FEE069F821884340210843E061F822105904229043F8221051201C90F7B2FF206800216DF720FF164A1378002B0AD0E06900043BD41A4880791A4A1178014001D1002831D1271C5C3739880023321CB7
:FB6B4200301C94F7D7FA3888FFF78DFE2E7008490E701048067022E0C0463C950900641B0800301B08005CC808005DC80800900608004D96090054950900B7C10800D020080060930900689309004C960900B6FC0000C49409004E96090001232B70201C28308DF7BDFDE069000407D48DF7DAFD8EF7AAF8012801D18DF7C9FDB7490E70A36B1B072FD5E06900042CD4B4494B681B0528D5201C01218EF77DF823E0B0490868800715D5F82210590821084310518021E069000400D44900AA4A11600120000779F75AF8002E0DD1201C8DF706FF09E0E069000403D5201C8DF7B2FF02E00123A1480370012002B0F0BC08BC184730B503685B019D49CD18043E
:FB6C3D001CFFF776FEE069000403D4201C00218EF744F820687CF7FBFEE0690006C00E0A2817D1012120688140934803688B430360201C74F710FFE069F821884340210843E061206884F733FA201CA030042102F034FB211C281C01228FF72BFFE069F821884318210843E061F82108590721084340218843F8210851206801218140CA437E490B6813400B606DF75DFDE069000403D47A480378012B03D05C342088FFF7B4FD012030BC08BC184700B5011C1D2079F759F808BC1847000070B5061CC169090417D4051CFC352C68002C03D0201CB6F7A8FB0AE014209AF7FDFB041E09D02860321C67490023B6F77DFB0C21201CB6F784FB70BC08BC1847A6
:FB6D3800F0B5071C0024614E0622151C6543391CA81902F0B5FA002805D1A8190621BEF737F9012003E00134042CECD30020F0BD70B5061C002529236B4355481C18A11C301C062202F09CFA002803D00135042DF1D310E0221C25329107890F01D1106808E0521AC9001368CB402020411A50688840184300E0002070BD30B500296FD000286DD0CA695205520F0270CA699204520F42704A6B831C9C07A40F01D11A6006E01A70120A5A70120A9A70120ADA708A6B831D9C07A40F01D11A6006E01A70120A5A70120A9A70120ADA70CA6B031C0A339C07A40F01D11A6006E01A70120A5A70120A9A70120ADA700A6C031C0E339C07A40F01D11A6006E01A89
:FB6E330070120A5A70120A9A70120ADA700C1C503422888274120AC274A3780375E3784375CB7B83758B7EC375CB7E03761A4A137843760D1C98352A68520F8276E289C276120A0277F4310968021C1D329007800F01D1116006E01170080A5070000A9070000AD07030BDC0465CC80800181B0800641B0800D45008005DC808007C290800E4C70800B4C408004C960900E96C09003C95090054950900C893090070B5002800D184E0002900D181E04A78D4000B785B075B0F1C43C3693F2212029343A206920C1343C3618C1CA3079B0F01D1226808E0E41ADB002568DD402022D31A62689A402A4342638C1DA3079B0F01D1226808E0E41ADB002568DD40EC
:FB6F2E002022D31A62689A402A4382630C1C0A34A3079B0F01D1226808E0E41ADB002568DD402022D31A62689A402A43C2630C1C0E34A3079B0F01D1226808E0E41ADB002568DD402022D31A62689A402A430264041C5034CA7C12028B7C1A4322804B7DE3700B7DA3708B7DC373CB7D83760B7EC3768A7E98263358DB00DB0852071343061C983633600A7F1202CB7E1A43E281F4300A1C1D329107890F01D1136808E0521AC9001468CC402023591A53688B402343036070BD10B5042810D22921414308484418002020706070A01C0621BDF7E4FF044A1188201C0830BDF7DEFF10BDC04654950900CA93090010B5AC4AAC4900780302AC4C20680004183C
:FB7029004308601078C3020868184308606068000423681B0C18434860507888600020C860012010BC08BC184710B5041C00290AD18EF7DBF870342078042815D19C484379012B11D10EE0022906D15030407F77F705F80023A38107E0052905D100F0E7F8002801D18DF7A1FE10BC08BC184770B5904D2B68FF2B56D1002077F7C8FD2860FF2850D001238B4803608B4803708B4C0323E3748B480168201C6FF705FC25232374022363743323A374201C7030042303700023437023632384824803685B006384242000230355E3818EF759FB286878F75BF87D4E30607368802003437360286877F7DAFF211C503103680B77C269C8680726B04332401043C2
:FB71240001225202104380221043C8600023CB750B6813430B6001238B7702234B776D496D488DF790FE201C6FF744FB012070BC08BC184770B5061C041C0023674803605F480378002B04D140235C490B60980527E04B0704D570342078042867D144E08B0724D5351C70352B78022B5FD16978564802685A4803684B43301C934213D95300638418360123737304232B703323A37400236B706FF7AAFD2023474E3360D80578F779FD42E0013169701EE0CB073DD5351C70352878022838D315D0042817D334D147490868430E47490B6047488DF72CFE02232B704823A37440490B685B006384183401236373301C6FF77FFD1DE01023314803601806784F
:FB721F00F74DFD334803685B00638418340123637304232B7000236B70301C6FF7C8FB35493548062202F038F8002802D133486FF7BEFB70BC08BC184731498868002805D0007C2438012801D8012000E00020704700B51D211C4802F03FF81921274802F03BF8FF23274A1360144A13600023264A1370FF23254A13608DF79CFD00BD10B583B0041C0C22E92109036846BDF76AFB694600200A7801312254174B1A5401300628F7D34B78A37103B010BD4D960900B8890E0038800E00A42C08008C060800D4500800BEC10800F0500800B00608009006080000820E00D85008006400080018800E009806080098830E00E4500800E0500800F8950900E8501C
:FB731A000800645108006C21080088060800BFC10800D893090000B500231E490B701E486FF787FB1E490868FF2804D077F70EFEFF231A490B6001231A4803601A480378012B04D18EF76CF9002316490B7000BD30B5041C051C70352B78022B18D1503076F7AAFB58231B5D022B11D1236D5B061B0F032B0CD10C4A1068410308D50721C904014004D10948FFF77CFF03232B7030BC08BC1847BEC10800F05008008C060800D4500800BFC108002C8B0E00C4940900F0B582B00C1C01D1042099E0051C4D480268002A08D0281CC4F764FA002803D0FF300006000E8BE0F82148590007800F012828D1E869000425D4237B5B0822D04149086880071ED528EB
:FB7415001C28308DF791FCF822505902229043F8225051201C9AF789F80821281C7EF7DDFF8DF7C4FA0123364A1370364A1168281C8DF7ABFA281C8DF7E7FBC0E72F687B0132481E18F37F012B50D0237B5B0809D1637B2E490091052B09D0DB002D48C218009204E0201C0C307BF7B3F8009000990B7963770023236001F03BFF01900099486840010BD4B068002805D003682360B3681C60B46011E0B46024600EE0F068002805D003682360F3681C60F46001E0F4602460211C281C90F7E5FB0123BB401549086818430860019801F01AFFE8690006C00E0A2803D1381C74F7FEFA09E0082807D1381C6DF7B1F903E0201C9AF71CF864E7002002B0F0BD3A
:FB751000BCC80800641B0800BFC10800885008007C290800589309006CCF05007429080070B582B00023019360490868202800D1B6E010285AD15E49086877F7BBFD051C5C4E301C77F7DEFA002811D0041CF822135801221343F8221350EB69C06907210B4088431843E061286877F7F4FC0CE02C1C311C281C28300622BDF7FBF9F820435902208343F8204351311C201C8DF741F9002805D0F820035901200343F8200351201C8DF718FB01F0A6FE012321688B40414A11681943116001F0A5FE20686DF755F8E369F820834310200343E361206801216DF7B9F9201C90F7F5F9201C8CF792FFFF233248036059E0FF23013398424AD12F4877F785FA04F5
:CD760B001E50D077F7F1FEE369012000068343F820834310200343E361E36C5B005B08E364EC210B59000683430B51201C00217BF769FF201C00217BF7C0FF6B4601AA211C4C31201C283096F7C0FD002806D0019B002B03D0201C7BF7B8FB03E0211C002078F79AFBFF231348036015480368012B18D1E3691B0415D412480368002B03D1114803680F4803608DF75CF80AE0402802D18EF734F805E001235B02984201D18DF7C5FF012002B070BC08BC1847C046D45008008C060800E8500800B4C4080088C8080088500800D0930900B6
:FB76F800A048002303608360704770B59E490B68180A9E4A402803D19D49D1609D4906E09D490143D160030219189C4BC9189C4D29609C4C9C4963685B0E2468E407E40F634009D0402807D17F2464020B68974D2B400125ED0406E0FD2424020B68934D2B400325AD040B600B682B430B6000238F4E336003040B21090459182143032631438C4E31600F30106070BD10B5041C7C480368002B05D1201C6FF71CF9201C00F096F810BC08BC184710B5041C8248416A002902D1836A022B09D9032904D1836AFF203630834202D2201C6FF75EFB60237A48195D405C80210143784A116070480368774A136043681720800603435360FFF78AFFA37B734A13AA
:FB77F300600023734A1360082113206EF7CEF910BD00B500290ED1FFF7CAFF5B4A11686D4841435A4A1068000A0430BDF7EDFC6A4A106014E0022907D1012368490B604030407F76F726FC0AE0052908D1002363490B60FFF707FD002801D18DF7C1FA08BC1847000000B5484A011C1368002B0DD09368002B0AD19389936060310A780023022A00D2531C0B706FF749FA08BC184700003D49037D022B07D10868431E00D30B608868431E00D38B60704710B5037D092B0CD14A4C4B4A106877F781FC20606068802188436060474AD078206210BC08BC184700B50821444800231A1C93F7AFFB00BDF0B5061C0F1C274C6368FF2B07D1012077F7A6F96060F8
:FA78EE00FF2801D1002041E03B4D0123EB742169281C6EF7E7FF2760A389A3602F4979431C480068000A0430BDF771FC2C49086024232B7402236B743123AB74281C6030002303700123437000238370C3702B625D2002234355606877F735FCA8730123EB73124F391C301C8DF788FA606877F72AFC391C6EF72BFE311C1C480622BDF70AF82169281C6EF7BCFF0120F0BDD493090094060800C8890E0040C07DC0447E000000D07DC0043E00008C800E00CC940900B88A0E00FFFFC3FF94830E0098830E006C210800A8060800A4860E0040820E0000830E00F8800E00710200009C830E00F0FC0E0000820E00D8930900F8950900B6FC0000645108005F
:FB7A3A00F0B5051C13235B049F4F3B60082105206EF7A8F89D4F3B689D4803403B603B68C00703433B608B4F3B6802273B43894F3B60974C984820620123974F3B60974FB868606278686065A8692430C17880220A43934F3A60934E8378B07B002B0ED1924D0021B0F7D1FDB169081C243042781302007B18430022B0F7DEFF09E00121B0F7C3FD8A4D8A4A13680120400603431360884805608848838A8848036000232360F0BD05238381836926331878012819D18348844A13680360834A11680161834A116841600022D343814A136000235360784A1368802003431360754A1368800403431360704700B5C369002B1CD013235B04644A13605A4A1344
:C97B350068584A1360564A1368544A1360504A13685F4A13606C48704A13680360704A116801616F4A1168416060486EF7AEFF08BC1847000030B5052383816A4A116806220A40062A02D181692A3108E08B0702D481692C3103E04B0704D481692E310B8801330B8013235B0448490B604F49CB69002B12D1514C2568C37B012B0CD1236880208343236002209AF7E6F880231D43A06899040843A060256030BC08BC184713235B04394803604048C369002B02D1424803680360704700B5002901D1FFF721FF08BC184700005A
:FB7D580000B52C22B049B148BCF710FEAF48B04B1860B0494160B049816100BD30B5041CBE342178FF233D334B43AC495918FF2208328B18FF211970A9493C30062201F08FFA00280CD1A74D23782B6002236B717F21C943A81D072201F08AFA00232B7130BD30B5041CBE342078FF233D3343439A495D18203083F78DF9281C6EF73AFE86F75CF99748036821788B4203D1FF2303600023437130BD00B5017D032901D0042902D1B2F7BFFF09E0037D062B02D100F008F803E0092B01D1B2F7E5FF08BC1847000070B582B0051C041C8034E37A002B08D0036DBE3319780820AFF724FA0023A376E3726378032B28D0A87B99F748FD4008218C431A1E04362C
:FB7E53000C618C00291DD08E421BD36078012806D1688CBDF7F1F9062803D13E2002E0042803D008202B6DAF33187003236370281C6EF7A3FD2B6DBE3319780520AFF7F6F931E06068002808D00090002301936946A87B99F76AFE002363606378032B11D0FF201930285A864209D8A87B86F78AF8002804D1281CB3F7C4FA002802D05B49C8780CE06378002B07D1594BA87B185C032802D25549887801E054494878A874281CB3F7A0F902B070BDF0B581B0041C051C80350027AF81EF76FF230533C618F37D0133F375C37B012B13D17378002B19D1484803689B0715D5A07B99F7D3FC80084100A06981420DD099F767FC4000686008E0012373703C4829
:BA7F4E000378A3740123DB07B361B7703B4800680090830739D539490B685B0602D40098430710D5A07B99F7B1FC400828846B78012B08D102236B70236D588900016884201CB2F7F8FFF37D012B05D17DF757FF011C201CAFF7EEF925484379022B14D1236DBE330068197888420ED17DF747FF1F4B991D1A7988541879411C0720BDF752F91A4B18711E4B1F7000980621014006293AD1236DBE33187886F727F8201CB0F77CFDF078012804D8164980000B5C01330B54E37B0099201CB3
:FB800800002B02D1B2F7E6FF01E0B3F712F8201CB0F71DFBAF7230E078E405000C95090078150800F17D0900FF7E0900349D080009C108000494090074150800E3C00800BC8B0E004015080086030800ECB00800B77583070AD5A87A0A490B78984205D2E37B002B02D00130A87206E02B7E002B00D02F76201CB3F796F801B0F0BC08BC1847C0461CCD0800F0B581B0051C0C1C08790002C978084350D00020ADF7A6FEFF2801D109234AE0071CADF760FE0023038121790902E27811438186C186051C83F7A9FB2E1CB03673885808E8806379252B0ED2384800900521BCF771FF6179C8084907490F01228A40009B195C11431954B07BFF233D334343309A
:FB8103004819180091281CB0F75CF82E488566B2F71CF9307B0021B0F793FA0523AB80381CB0F7DEF800999E3101200870381C002100F035F8A279E179381C00F005F801E012232B7001B0F0BDF0B50C1C171CADF710FE061C201DB4F7EFFE051E1ED0B18D0B051B0D012040031843210408432B1CA907890F01D1186006E01870000A5870000A9870000AD8703A06120E2104090C281D91F76BFC281CB3F75AFAF0BD30B50C1CFF233D3343430548C51801F0AAF8A2352C8001F0AEF830BDC046F44E0800349D080038B00800F0B5061E20D00768002F1DD0407CADF7CCFD051C707C182141430C484418786891F76BFA99F7ECF9381C99F7A3F900233360A3
:2281FE00217A01312172217A05480278A88D91F7A0F900232372F0BDC046F4B008007C15080097
:80822C0070B5051C0E1C041C8034A37F002B1ED0B0F76FFD184A537C012B09D9E37E002B02D1A08BC10603D5311C281CB0F734FDCD23585D00280AD0FF230533E818837D002B04D04378002B01D1012383700B490B681B070FD56378022B0CD1FF201630285C002807D0A0898004800E0023002800D10123237670BDECCC0800E02C0800F1
:FB82B400F0B5041C051C3A4806689835A8880712F306D90FE9707307D90F0307DA0F002F04D0344803685B0300D5111CFF231533E0184378002B03D1002901D0012343708A4216D0AB79002B15D1002F08D0D0231859C168C91BC16002D48368DB1983600122AA71201CB3F785F8201CB0F778F801E0002383713307DA0FA8884307D90F8A4234D11C4F397C0A0702D5B304990E2DD1184A13689B0303D5B3079B0F032B25D004214840A880251C5035AE87B304980E1CD020221149BB68181D00F0DAFFCC342078800712D50D490B68012080030340580B0BD02B68BE331878ADF7F1FCAF303D210170012028870023AB87F0BDA88B0E00E02C0800ECCC0881
:9583AF000080980E00BC8B0E0010B51F4C2068002805D08008800099F7BBF80023236010BDF0B5051CC668B469002C16D0B0F72FFE002812D1154F3A1C211C1331E01CB0F707FD381C00F00AF80023AB60EB60A008800099F79DF80023B361F0BD00B582B0262369460B800190081C77F721FC02B000BD00B54368002B04D010220448002192F700FE00BDC046E49C08000996090017200000AF
:9C846000F0B583B00291FF233D3343432248C618356D00F049FF371C90372C1CB0348E239A5B02998A1A1204120C638853433A6FD21851014909019100F03EFFF37B012B0ED16B8B5B000093288B4000019A101841014909181CBCF7BDFEA0800098E080281C83F7ACF9F37B002B0ED1E68870086883A188019899F79BF9E288011C101CBCF7A8FE301A400828830298431E3B800123BB7203B0F0BD349D080089
:EC850400F0B581B00090ADF734FC041C0027344E336BDB071FD5B4421DD0251C2C354223A97D9A5D914216D1291C1031301C3C30062200F0BFFE00280DD100F0E3FE051CBE36307800F032F8281C00F0E3FE3078AFF7EAFE03E0C03601370F2FD8DB0098B3F73BF8251C0123EB852C35201C81F723FB00980021AEF723FD1A4A13681021DB0603D5A971201CB3F7AFFE201CB2F76DF8BE342178FF223D325143124BC9187F23FF2023300B5401B0F0BD10B5FF233D3343430C48C418201C80304178012907D1418C608CBCF73FFE062803D13E2002E0042903D00820236DAF33187010BD2890080040150800349D080048
:BC85F800F0B5061C046D2B4803689E4201D1B0F787FD301CB0F7C3FB351C8035288901380ED32881288904236B70002808D1301C6EF7D1F9BE3421780520AEF725FE38E0687800281FD1B07B99F74BF94008B034A16899F7E1F801239B0698420CD267883B1859014909381CBCF7CCFD7843A168081840014009A060A06800236B700223F374B06112E0022810D1AB7E002B0DD0E889298A431A1804000C074B984205D2EB7A002B02D1301CB2F71BFD301C6EF734FBF0BD6C210800FF7F00001F
:8C86F000F0B5051C1F49FF230533C418E378980000230B544318581C00230370AF692B6D1889421C267C688C5043B04063681B1858014009381A01239B06984220D2B31D20789840A368D901EB7B002B00D15143E268824200D3101CBCF758FD011C802800D980219F352970074803789E4202D2701C207404E000230434191C381C0BC4F0BDC046ECB008006F15080081
:E4878800F0B5061C071C9C373888102101401D490BD01D4BF518EB7898000A5C9301AA68D218AA604318597811E0174BF518EB7898004118487800280DD08C78097861438901BCF717FDA9680918A960211C8B01E868C018E8602B7C002B11D1E86800280ED0AB68D901F37B002B03D1336D1A8901325143BCF7FEFC802800D98020F870F0BDC046ECB0080004010000F0B50D1C114C20600B68DB0701D598F7F4FF0F4E0020706637680E483840306099F700FB99F7FEFA2868E0606868A0600220706699F7F6FA99F7F4FA99F7F2FA37600020E060A060F0BDC04600820E001C800E00FFFFFFFD2F
:3088740000B54068084A13681979002909D1074A13681B0605D4002801D098F757FE012000E0002000BDC046C04F0800E02C080063
:7888C00030B5041C80304378002B1BD10323E374252101230B55837E002B07D0236DD98B09014184A36903840123C372618CA06975F70EFA238C984204D02084216DB03188800880FF230133E158E518A06998F77FFF216DB2310A88011C101CBCF76EFC011C201CB2F7C2FCA3692B60201CB0F7D0FB00236B7130BD5A
:FB894800F0B581B02F4806682F4805682F480378002B52D12E480368AB4203D12D480368B3424AD02C4C2D4FFE20284007D1002D03D02B480368DB0301D5002E1CD063681B071B0F022B02D0022099F7D5FA25480078606324480078A06367F753FC00F0C7FC822141432068642250436430BCF721FC431C3B6018E063681B0702D0002099F7BAFA00206063A063184A13680093174A1088392109014143181CBCF70AFC386014490098BCF705FC134908603868A06107490D6007490E6001B0F0BC08BC1847C04614CD0800B4C4080008C30800B8CA0800F49309000C000F00DC5E0800FC0A080009C308000AC30800C02D0800E80A080020CF01009C000F40
:FB8A430000381CFFF795F902B0B1F782FEFFF7B3F9B1F78FFEF0B5041C00216EF716FD002803DA01234D4843716FE0061C251C7835687A00280DD1A07B98F72DFF4008236DB833196898F7C9FE002804DC687A002805D0002E03DD201CB2F787FB55E0E37B012B03D1002801D101236B72A878802101433B4A1160082105206DF76EF8374A5379002B41D1B0F725FB364F381C052100F010FC03233B74201C00F037F8B0F7D6FAEB8A002B0AD1FF201630205C002805D1B0F70FFB3B7C082003433B740023AB74FF230533E6180023F375201CB2F752FC254A13780021002B00D101211170F078FF2806D16B7A022B03D1081CF070A3697360012805D8F17031
:7E8B3E008B001B48C0187B7C8370201CAFF777FCF0BD30B5847C17490B788374051C012200216EF733FBAC742C6DB223195B0239884200DB081C10494143E5208000BCF73EFBFF210531695C884200D3081C32342178490702D5012800D901200349487430BDA42C0800A4860E00ECCC08006C150800ECB008007415080071020000E1
:FB8D080003490B680020012B00D101207047C046901C0800002E02D00020E05504E0E35D002B01D0013BE3557CF71FFF10B5A24C201C042100F0DCFA7F21C943A01D072200F0BEFAFF23236000239C4803709C4803709C4803709C4803709C4803709C4B9C4803600123DB029B48038080239B48037000239A4803709A4803709A480621BCF71EF914219948BCF71AF914219848BCF716F910BD30B5041C96480368002B04D000230360282300201855924D00216962A96278F7F7FD90480368002B03D176F764F9002803D1012091F731FE04E077F797F82834042020700023884A137088480378012213430370FFF79FFF281C8A300621BCF7E4F830BDF0C2
:FB8E0300B5061C051C081C08356C4C2368FF2B20D076490330062200F04DFA002819D16079022807D12068ACF7A4FFC38D012B10D1002711E001280FD1206876F741F9C1690906C90E0839062903D2FF210931475C02E0122333700EE0A11DE81D0722BBF78FFD8021A01D072200F02CFA00232371AF710823F370F0BD30B50C1C5B4D0331281C0622BBF77CFD637A564803701422211C0A315648BBF773FD1422211C1E315448BBF76DFD002347480370434CFF232360281C0021ACF765FF002803D1281C0121ACF75FFF002806D0C38D012B12D1BE30007802210CE0281C75F719FE002809D0C2691206D20E083A062A03D2006801212060617130BD0B7963
:FB8EFE0035480370CB78304803707047F0B5052630480378002B50D12A4C2768FF2F4CD02079811D0720BCF7A6F905062D0E607902280CD1381CACF71FFFC38D012B3CD1A31DEA560024012622490E7016E0012833D1381C76F7B7F8C1690906C90E0B1C083B062B29D2A31DEA56FF230933C45C0123174803700A2900D10326144800211D4B1B579A420DDA0278013202700278B24212D301700F4A1378002B0DD092F7BDFB0AE0154B1B5701709A4205DD06480378002B01D092F796FB0120F0BC08BC18470494090002C108000FC10800840308008603080010C10800C05D00009C070800A007080099070800D8C20800ADC9080009C1080011C108002593
:FB8FF900C1080024C9080054200800DCCC0800EEC00800E00A0800381CFBF7A1FE6BF7B2FB281CFBF7BAFE6BF7CBFB81B000F003F874F7ECFD0000F0B5041C0D1C7CF709FF324E7379012B12D180213368095D8B420DD1A02210553179891988713079411C0720BCF70AF930710023284A1370271C261C6436317F9F2038569F377CF798FE3870371CB37D0C37002B15D03368DB0508D41F4803691B010ED5301C90F773FE002809D00023B3610123FB720023BB727B72301C8EF798FE33685806000F295C002904D0144B185CB072431E0DE010490B69DB000BD5104A11680A6853031B0F984204D193025B0F013BA3810CE0012333723B68FF20013083434F
:2890F4003B600D2307490B70301C74F715FEF0BD0494090086030800542008009EBB05001C2B0800E8C008003C
:5491440083780D2B02D1032311480360704700B50F480368002B05D0002303600D21181C7AF79AFC00BD00B5094902060CD40868012807D102230B6018220D2100207AF76AFC03E0032801D1022000E0002000BDF09309007B
:1891B400044A1088012149020140480A012250407047C046E8C4080099
:FB922C0000B500F06BF800231D490B7000F06EF800BD00B51B4B984202D1081C00F001F800BD00B5012100F006F800BD00B5002100F001F800BD30B50D1C114C12490B78012B15D10178032901D0082910D18378002B0DD100F042F8002D03D023780133237003E02178013900D3217000F03EF830BD00B5FFF7DAFF00BD01490878704754960900B8520800540008007847000000C09FE51CFF2FE1FC4005007847000000C09FE51CFF2FE1CC4805007847000000C09FE51CFF2FE1E05105007847000000C09FE51CFF2FE1741005007847000000C09FE51CFF2FE1304F05007847000000C09FE51CFF2FE17CD704007847000000C09FE51CFF2FE190D70434
:CD932700007847000000C09FE51CFF2FE160E801007847000000C09FE51CFF2FE1CC510500910000000B8F090092000000000000000000000003000002000000000000000000000000000000000000000000000000000000009551020053700900597109006B7309000000000000000000000000006754020000000000A1780900000000000000000005780900857709000000000059780900000000008778090087510200010021000C0019000200000000180000FF00000080020000800200009C93090000180008030000000100000093
:00000001FF
